S02000006F70656E626C745F6F6C696D65785F73746D3332703130332E7372656307
S315080000000050002079060008510600085506000829
S31508000010590600085D060008610600080000000091
S31508000020000000000000000000000000650600084F
S3150800003069060008000000006D0600087106000841
S31508000040C1060008C1060008C1060008C106000866
S31508000050C1060008C1060008C1060008C106000856
S31508000060C1060008C1060008C1060008C106000846
S31508000070C1060008C1060008C1060008C106000836
S31508000080C1060008C1060008C1060008C106000826
S31508000090C1060008C1060008C1060008C106000816
S315080000A0C1060008C1060008C1060008C106000806
S315080000B0C1060008C1060008C1060008C1060008F6
S315080000C0C1060008C1060008C1060008C1060008E6
S315080000D0C1060008C1060008C1060008C1060008D6
S315080000E0C1060008C1060008C10600080000000095
S315080000F000000000000000000000000000000000F2
S3110800010000000000000000005FF808F195
S3150800010C10B5054C237833B9044B13B10448AFF337
S3150800011C00800123237010BDE001002000000000C0
S3150800012CF04F000808B5034B1BB103490348AFF35E
S3150800013C008008BD00000000E4010020F04F000814
S3150800014C02F078B902F088B908B5054B9868C0432F
S3150800015C10F0010000D108BD00F0CAF8012008BD56
S3150800016C00080140642000F093B800BF00F096B870
S3150800017C00B5C7B0002168464FF48C7204F01CFF1A
S3150800018C6946094804F086FD50B9009828B19DF8CF
S3150800019C080080F01000C0F3001047B05DF804FBAF
S315080001AC002047B05DF804FB18500008004870475B
S315080001BC18500008002310B5064C0A22204606499A
S315080001CC84F8283204F0B6F910B9012384F82832D9
S315080001DC10BD00BFFC0100200850000838B50D48BA
S315080001EC90F82832012B11D002F0CCF80A4C00F109
S315080001FC640503E002F0C6F8A84202D823685B0639
S3150800020CF8D50648BDE8384004F072BD04F07EFC0B
S3150800021CEAE700BFFC010020004400401850000823
S3150800022C034890F82832012B00D0704704F06EBCB6
S3150800023CFC01002070B5144C064694F82832012BA4
S3150800024C16D033789BB1114C636002F09BF800F121
S3150800025C0A0505E002F080F902F094F8A84202D8E3
S3150800026C23681B06F6D516F8013F002BECD170BD9A
S3150800027C214604F0BDFD0028E3DA0023204684F865
S3150800028C283204F043FCDCE7FC0100200044004063
S3150800029C014B1880704700BF2804002010B502F0E7
S315080002AC71F80F4C236898420ED30E4B1A7862B12C
S315080002BC00204FF480510C4A1870116102F062F854
S315080002CC0A4B1B881844206010BD01204FF480513E
S315080002DC02F1804202F5883218705161EEE700BFD0
S315080002EC2C0400202A0400200010014028040020B9
S315080002FC4FF48052014B1A61704700BF0010014041
S3150800030C234908B50A460B6823F0070343F0020392
S3150800031C0B60136803F00703022BFAD11D4B1A4620
S3150800032C196841F48031196013689903FCD5516832
S3150800033C184B21F47C1141F4E8115160116841F015
S3150800034C807111601A689201FCD55968114A21F01E
S3150800035CF0015960596821F4E06141F480615960F3
S3150800036C596821F460515960596821F0030141F02C
S3150800037C02015960536803F00C03082BFAD106489E
S3150800038C01F06CF8BDE80840002000F0A5B900BFE4
S3150800039C002002400010024000A24A0400242DE965
S315080003AC8048042793B000F0BBF9FFF7A9FFCDE905
S315080003BC0D444C4D0F94AB694FF4805140F2011229
S315080003CC43F020034FF001080326AB61AB69DFF855
S315080003DC1CA103F020030293029BAB69DFF8109172
S315080003EC3B43AB61AB69DFF80CB13B400393039B12
S315080003FCAB693D4843F00803AB61AB6903F00803EE
S3150800040C0493049BAB6943F01003AB61AB6903F02F
S3150800041C10030593059BCAF81410C9F810100BA9FC
S3150800042C0B920C9700F098FE0BA950460E94CDE94A
S3150800043C0C86CDF82CB000F08FFE02230BA948468B
S3150800044CCDE90D34CDE90BB800F086FE40F2044C2C
S3150800045C0922CDE90B44CDE90D44CDE90F44CDE98C
S3150800046C09441194EB6906A943F40033EB61EB6973
S3150800047C1D4803F400330093009BAB693B43AB6107
S3150800048CAB69CDE906C23B400193019B089600F087
S3150800049C63FE40F6080306A91348CDE9063700F0B3
S315080004AC5BFE0C234FF4E132A5F5E6350BA928467D
S315080004BC0F93CDE90C440E94CDE910440B9200F041
S315080004CC73FF2B6923F490432B616B6923F02A0382
S315080004DC6B61EB6843F40053EB60FFF731FEFFF7F3
S315080004EC31FEFCE70010024000080140000C0140F8
S315080004FC0010014010001004104B82B09969104A84
S3150800050C41F001019961996901F001010091009985
S3150800051CD96941F08051D961DB6903F080530193A5
S3150800052C019B536823F0E06343F080635360536880
S3150800053C23F0E063536002B0704700BF001002401E
S3150800054C00000140002310B501681E4A86B091428E
S3150800055CCDE90233CDE9043301D006B010BD4FF412
S3150800056C807403F1804303F50433DA6902A942F077
S3150800057C0072DA61DA69144802F000720092009A85
S3150800058C9A6942F008029A619B69029403F008037F
S3150800059C0193019B4FF4007400F08CFC0222032398
S315080005AC02A90948CDE90242059300F083FC074AE3
S315080005BC536823F4C04343F0E06343F48043536029
S315080005CC06B010BD00640040000C0140000001405C
S315080005DC08B500F05BFE164800F066FD154800F0FD
S315080005EC63FD154800F060FD144B1549DA6922F0D5
S315080005FC0072DA61CA6822F40052CA60DA6922F417
S3150800060C0032DA619A6922F010029A619A6922F02C
S3150800061C08029A619A6922F004029A61DA6922F050
S3150800062C8052DA619A6922F001029A6108BD00BF0C
S3150800063C00100140000C0140000801400010024067
S3150800064C00440040704700BFFEE700BFFEE700BF4E
S3150800065CFEE700BFFEE700BF704700BF704700BF4C
S3150800066C704700BF00F06EB8704700BF002103E06A
S3150800067C0B4B5B58435004310A480B4B42189A42B1
S3150800068CF6D30A4A02E0002342F8043B084B9A4286
S3150800069CF9D3FFF7E9FF04F04BFCFFF77FFE704731
S315080006AC4458000800000020E0010020E00100206A
S315080006BCA0110020FEE7000010B54FF0FF32002411
S315080006CC044BDA601C61DA60DC60FFF781FF2046B8
S315080006DC10BD00BF0010024038B54FF47A730D49AF
S315080006EC0D4A09781268B3FBF1F30546B2FBF3F031
S315080006FC00F096FA08B90F2D01D9012038BD044629
S3150800070C024629464FF0FF3000F054FA034B2046B8
S3150800071C1D6038BD040000200000002008000020E1
S3150800072C074A08B51368032043F01003136000F05A
S3150800073C2FFA0020FFF7D0FFFFF7DEFE002008BDDA
S3150800074C00200240034A044B11681B780B441360C3
S3150800075C704700BF781100200400002000287DD0C7
S3150800076C90F8203070B50446002B74D022681368B4
S3150800077C23F00203136001F013FE054604E001F0B2
S3150800078C0FFE401B0A285DD823685A689107F6D4D1
S3150800079C1A6842F001021A6001F002FE054604E0EE
S315080007AC01F0FEFD401B0A284CD823685A68D2076C
S315080007BCF6D5227E0025012A1A684FF001060CBFD1
S315080007CC42F0800222F080021A60627E012A1A68C0
S315080007DC0CBF42F0400222F040021A60A27E012AA7
S315080007EC1A680CBF42F0200222F020021A60E27E40
S315080007FC012A1A680CBF22F0100242F010021A6085
S3150800080C227F012A1A680CBF42F0080222F008025D
S3150800081C1A60627F012A1A680CBF42F0040222F0A1
S3150800082C04021A602169D4E9022002430A4360696A
S3150800083C6168024301390A43DA612846656284F81D
S3150800084C206070BD0522636A012043F4003363629D
S3150800085C84F8202070BDFFF775FE87E701207047E6
S3150800086C90F820300246013B012B05D9536A01202A
S3150800087C43F4802353627047F0B401244869136823
S3150800088C00F01F0204FA02F2D543D3F80042CE69EF
S3150800089C44F00104C3F80042D3F81C422C40C3F8B8
S315080008AC1C42A6B3012E13D18E8803EBC00408682C
S315080008BCD3F80CC28F6846EA004688894CEA020CC3
S315080008CC40EA0740C3F80CC2C4F84062C4F84402B4
S315080008DC886998BBD3F804022840C3F8040208694F
S315080008ECA0BBD3F814022840C3F81402096A0129DC
S315080008FC04D1D3F81C120A43C3F81C22D3F80022DD
S3150800090C0020F0BC22F00102C3F800227047CC6824
S3150800091C8E88D3F80C72D1F808C046EA04460C88BF
S3150800092C03EBC0002F4044EA0C44C3F80C72C0F821
S3150800093C4062C0F8444288690028CBD0D3F8040238
S3150800094C1043C3F8040208690028CAD0D3F8140265
S3150800095C1043C3F81402C9E738B590F82030012BB8
S3150800096C06D00123426A42F400224262184638BD78
S3150800097C0223026880F820301368044623F001032A
S3150800098C136001F00DFD054604E001F009FD401B5E
S3150800099C0A2807D823685B6813F00103F5D163624C
S315080009AC184638BD0521626A012342F40032626298
S315080009BC84F82010DAE700BF70B490F82040056878
S315080009CC013C012CAE6807D90122436A43F4802303
S315080009DC4362104670BC704716F0E05F2FD0C6F322
S315080009EC0166032E33D00120B04018608B68A3BB78
S315080009FC0C68C86806F1180340EA44501B01E85015
S31508000A0C0869097D3601AB190129C3F8840105D19A
S31508000A1CD3F8841141F48071C3F8841151683544B4
S31508000A2CC5F88C1111680022C5F88811D3F8801105
S31508000A3C104670BC41F00101C3F8801170470122C1
S31508000A4C70BC436A43F40013436210467047436A0A
S31508000A5C012243F400034362BBE7C8684C680343AE
S31508000A6C06F1180043EAC40300012B50C8E700BF7F
S31508000A7C90F82030013B012B01D900207047036800
S31508000A8C89069B6831EA030314BF012000207047CE
S31508000A9C2DE9F04190F820500446013D012D06D968
S31508000AAC0120636A43F480236362BDE8F08105681C
S31508000ABC002958D02869800758D008012E18D6F86E
S31508000ACCB07107F004079760002F5CD1D6F8B071A7
S31508000ADC7F0D1760D6F8B0E10544D6F8B4C1D6F840
S31508000AECB471D6F8B461D5F8B8810EF0020E0CF0D4
S31508000AFC0F05C7F30727360CC2E903E5C2E90567F4
S31508000B0C83F8008022680244D2F8B821120A5A7077
S31508000B1C22680244D2F8B821120C9A702268024450
S31508000B2CD2F8B821120EDA7022680244D2F8BC2127
S31508000B3C1A7122680244D2F8BC21120A5A71226828
S31508000B4C0244D2F8BC21120C9A7122681044D0F8CF
S31508000B5CBC21120EDA71226879B9D368084643F0BB
S31508000B6C2003D360A1E7E8688607A6D1636A01204B
S31508000B7C43F400136362BDE8F0811369002043F067
S31508000B8C2003136191E7D6F8B071FF085760A1E707
S31508000B9C4FF6FF01064A0002D36800F4E0600B40EA
S31508000BAC43F0BF6343F400330343D360704700BF7D
S31508000BBC00ED00E0184B30B4DB68C3F30223C3F135
S31508000BCC0705042D03F1040428BF0425062C19D99E
S31508000BDC4FF0FF34033B9C4022EA04044FF0FF32EB
S31508000BECAA4021EA020101FA03F222431201002863
S31508000BFCD2B20ADB00F1604000F5614080F80023B0
S31508000C0C30BC704700242346E8E7044B00F00F007D
S31508000C1C03441A7630BC704700ED00E0FCEC00E0AB
S31508000C2C0138B0F1807F0DD230B4F02500220721AF
S31508000C3C054B064C586084F82350104630BC9A6015
S31508000C4C196070470120704710E000E000ED00E0E5
S31508000C5C124BDB6813F0100305D010231049CA6930
S31508000C6C42F00202CA610D4AD268500706D50C49F1
S31508000C7C43F00403CA6942F00102CA61074AD16902
S31508000C8CC90708D50648C16941F00401C161D16993
S31508000C9C21F00101D161014AD3607047002002405E
S31508000CAC80110020064B186910F0800006D0054903
S31508000CBC054A59605A601869C0F3C010704700BFDE
S31508000CCC0020024023016745AB89EFCD034A00207B
S31508000CDC136943F080031361704700BF002002407C
S31508000CEC70B5054601F05CFB134C064601E06A1C20
S31508000CFC12D1E368DB07FAD4E368980644BF2023CD
S31508000D0CE3600D4BDA68D10602D4DA69D2070BD543
S31508000D1CFFF79EFF012070BD25B101F041FB801B3A
S31508000D2CA842E6D9032070BDD86810F00400F2D0AA
S31508000D3CFFF78EFF0120EEE7002002402DE9F04F69
S31508000D4C274E0746307E83B0012843D09A460123A6
S31508000D5C4CF250300D4690463376FFF7C1FFA0BBD8
S31508000D6C012F3BD0022F0CBF0223042301934FF013
S31508000D7C000B5F46DFF86C904FEA0B14C4F12001A8
S31508000D8CF7610AFA01F128FA04F2203C0A432AFA16
S31508000D9C04F4D9F81010224392B241F00101C9F8B3
S31508000DAC10104CF250302A80FFF79AFFD9F8102011
S31508000DBC0BF1010B22F001025FFA8BF10235C9F82F
S31508000DCC102010B9019B8B42D6D80023337603B07A
S31508000DDCBDE8F08F022003B0BDE8F08F0197C6E797
S31508000DEC80110020002002402DE9F843DFF8C0905E
S31508000DFC99F81830012B56D0012203680646022BA7
S31508000E0C884689F818204CF250302FD0FFF768FF27
S31508000E1C78BB4FF0FF33C8F80030D6E9025305EB20
S31508000E2C83239D4225D20746204C07E0D6E9023299
S31508000E3C05F5806503EB8223AB421BD9C9F81C70F8
S31508000E4C23694CF2503043F0020323616561236930
S31508000E5C43F040032361FFF743FF236923F00203A2
S31508000E6C23610028E2D0C8F8005003E0FFF738FFEA
S31508000E7C28B10120002389F81830BDE8F8830B4CFB
S31508000E8CC9F81C0023694CF2503043F00403236163
S31508000E9C236943F040032361FFF722FF236923F0FC
S31508000EAC04032361E6E70220BDE8F883002002402C
S31508000EBC801100200A68002A00F0DC802DE9F04F2A
S31508000ECC4FF0000A85B05546DFF8D0C1DFF8D0E1FF
S31508000EDC6D4FDFF8D08103E0013532FA05F379D08E
S31508000EEC0123AB4002EA0304A342F5D14A68122A4D
S31508000EFC00F09F8000F28880022A00F09E807DD93F
S31508000F0C032A6AD0112A02D1CB6803F1040AFF2CF2
S31508000F1C67D881460368AA000F2606FA02FB23EA5D
S31508000F2C0B030AFA02F21343C9F800304A68D300D5
S31508000F3C62D5DCF8189025F0030349F00109CCF8C2
S31508000F4C1890DCF8189003F1804309F00109CDF8E4
S31508000F5C0C9003F5803305F00309DDF80CB04FEA65
S31508000F6C8909D3F808B006FA09F62BEA060670457D
S31508000F7C019611D0404564D0444EB0427BD0444EC5
S31508000F8CB0420CBF4FF0030B4FF0040B019E0BFA4B
S31508000F9C09F946EA09060196019E9E603B68D60346
S31508000FAC4CBF2343A3433B607B6896034CBF234348
S31508000FBCA3437B60BB68D6024CBF2343A343BB60E9
S31508000FCC9202FB6815D51C43FC600A68013532FA97
S31508000FDC05F385D105B0BDE8F08FFF2C4FF0000A5C
S31508000FEC97D905F18042083A4368920000F1040942
S31508000FFC92E723EA0404FC600A686DE7A2B1012AA9
S3150800100C85D1D1F80CA082E7224EB2420CD020D959
S3150800101C214EB24208D006F58036B24204D0A6F567
S3150800102C8016B2427FF473AF8A68E2B94FF0040AAD
S3150800103C6DE7CB6803F10C0A69E7CB6803F1080A7C
S3150800104C65E74FF0010B0BFA09F946EA0906019612
S3150800105CA2E7A6F58016B242E6D006F58036B2426D
S3150800106C7FF455AFE0E7012A0CBF036143614FF0EB
S3150800107C080A4CE770474FF0020B019E0BFA09F968
S3150800108C46EA0906019687E700040140001001406C
S3150800109C001401400000211000003110001002401D
S315080010AC00080140000C0140264B98420DD0264BF7
S315080010BC98422ED0254B984213D0254B984234D0C3
S315080010CC244B984219D00120704703F58433DA680B
S315080010DC002042F00402DA60DA6822F00402DA60D0
S315080010EC704703F58033DA68002042F01002DA60A4
S315080010FCDA6822F01002DA60704703F57843DA688A
S3150800110C002042F04002DA60DA6822F04002DA6027
S3150800111C704703F58233DA68002042F00802DA6079
S3150800112CDA6822F00802DA60704703F57C43DA685D
S3150800113C002042F02002DA60DA6822F02002DA6037
S3150800114C704700BF00080140000C01400010014028
S3150800115C00140140001801402DE9F0470F68C7F349
S3150800116C0F2797FAA7F6B6FA86F637FA06F36ED06D
S3150800117C4FF0010C4FF00F0E4FF003084FF0040A16
S3150800118C56E040F20113B340C2684FEA132999FAA4
S3150800119CA9F4B4FA84F50C6922EA0902AC40224394
S315080011ACC2601C0E93FAA3F5B5FA85F593FAA3F269
S315080011BCB2FA82F2AD004FEA820902590EFA05F527
S315080011CC22EA05054A6802FA09F2154305514A68E6
S315080011DC22F00802012A27D193FAA3F2B2FA82F274
S315080011EC93FAA3F9B9FA89F9920008FA02F225EAF0
S315080011FC02058A684FEA890902FA09F22A4302515A
S3150800120C93FAA3F9B9FA89F993FAA3F3B3FA83F320
S3150800121CCD684FEA89099B000AFA09F922EA0902FC
S3150800122C05FA03F313430351013637FA06F30ED0C6
S3150800123C0CFA06F33B42F7D0072EA2D94FF001124F
S3150800124CA6F1080302FA03F343F080639CE7002037
S3150800125CBDE8F0870A4A536803F4803373B15368C0
S3150800126C0848C3F340430133B0FBF3F0044B5B6807
S3150800127CC3F38343023300FB03F070470248F5E7D8
S3150800128C0010024000127A0000093D00164B1A465F
S3150800129C196841F00101196013689B07FCD553685E
S315080012AC114923F0030353604B6813F00C0FFBD161
S315080012BC0B680D4A23F080730B60136813F00073E8
S315080012CCFBD153601168184621F45021116011683E
S315080012DC21F0F80141F0800111609360536A43F0E4
S315080012EC80735362704700BF00100240114B10B553
S315080012FC5B68014603F00C03082B19D1FFF7AAFF0C
S3150800130C0C4B08605A680C4CC2F30312A25C0B4CCB
S3150800131CD04048605A68C2F30222A25C20FA02F254
S3150800132C8A605B68C3F3C223E35CD840C86010BD0F
S3150800133C0348E5E7001002403850000848500008FA
S3150800134C00127A00026812F040022AD1F0B4D1E9F0
S3150800135C0035044688682B43CD68034308692B433C
S3150800136C4D698E690343CF6920682B4333430E6A54
S3150800137C3B4320F47F40334320F0BF0003432360F4
S3150800138C6368B6F5005F23F0040343EA154363600C
S3150800139C02D0F0BC104670478B8C10462361F0BC0B
S315080013AC70470120704700BFC3689B0401D5012014
S315080013BC704730B504460D46C2684B6822F4B052E5
S315080013CCD1E90301034322F00C020B431343E360F8
S315080013DC2369AA6823F440531343236163696A6932
S315080013EC23F44073134385B063616846FFF77EFFA9
S315080013FC164B9C4227D0164B9C4205D0154B9C424B
S3150800140C02D0012005B030BD029B002BF9D02A680A
S3150800141C002AF6D003EB8303920003EB8303B3FB9A
S3150800142CF2F364210C4D0020A5FB03C2520901FB03
S3150800143C12331B013233A5FB0313120102EB5312B1
S3150800144C92B2A260DEE7039BDFE700BF00380140DB
S3150800145C00440040004800401F85EB51014B1860C2
S3150800146C704700BF0000002070B50B4D287300F0C4
S3150800147C89FF00F1320605E001F06EF800F082FFF4
S3150800148CB04206D8AC6814F00104F5D0E868C0B2CE
S3150800149C70BD204670BD00BF0038004038B500F05E
S315080014AC71FF00F5FA7503E000F06CFFA84209D24B
S315080014BCFF20FFF7D9FF044601F04EF8FF2CF3D1B5
S315080014CC012038BD002038BD70B54FF48056094D43
S315080014DCFF206E61FFF7C8FFFFF7E0FF10B101248C
S315080014EC204670BD04462E61FF20FFF7BDFF20463F
S315080014FC70BD00BF000C014070B50E4601060446CF
S3150800150C41D44FF48052254BFF201A61FFF7ACFFEC
S3150800151CFFF7DAFFC0B144F04000FFF7A5FF300E25
S3150800152CFFF7A2FFC6F30740FFF79EFFC6F3072097
S3150800153CFFF79AFFF0B2FFF797FF44B1082C19D1C1
S3150800154C8720FFF791FF05E0FF25284670BD9520FB
S3150800155CFFF78AFF0A24FF20FFF786FF054600F0EF
S3150800156CFBFF2A0604F1FF33EFD513F0FF04F2D183
S3150800157C284670BD0120FFF777FF0C2CEAD1FF2017
S3150800158CFFF772FFE6E700213720FFF7B5FF0128C2
S3150800159C0546DAD804F07F04B3E700BF000C014017
S315080015AC38B5841C00F2022514F8020CFFF75CFF10
S315080015BC023414F8030CFFF757FFAC42F4D1FF20A2
S315080015CCFFF752FFFF20FFF74FFFFF20FFF74CFFF7
S315080015DC00F01F00A0F10500B0FA80F0400938BDF4
S315080015ECF8B505460E4600F0CDFE00F1640703E09B
S315080015FC00F0C8FEB84222D2FF20FFF735FF04469A
S3150800160C00F0AAFFFF2CF3D0FE2C18D10235FF20D0
S3150800161CFFF72AFF05F8020CFF20FFF725FF05F850
S3150800162C010C00F099FF023E05F10205EFD1FF20EF
S3150800163CFFF71AFFFF20FFF717FF0120F8BD002060
S3150800164CF8BD00BF60B92DE9F047AA4F96B03D78B2
S3150800165C15F0020506D03878C0B216B0BDE8F0878A
S3150800166C0120704702264FF0010AA34BDFF8A0921F
S3150800167C9A69A24C42F008029A619A6902A902F088
S3150800168C08020092009ADA69484642F48042DA6106
S3150800169CDB694FF4805803F480430193019BCDE931
S315080016AC03A602940595FFF757FD09230322C9F8EB
S315080016BC10800393924B02A948460492029305950F
S315080016CCFFF74AFD04228F4B02A94846CDE90232A0
S315080016DCFFF742FD4FF482704FF40071382207234E
S315080016EC894C0D90119120460CA9129215930C95C4
S315080016FCCDE90E551095CDE91355FFF723FE236852
S3150800170C824A43F0400323604846C9F8108007A96B
S3150800171CCDE908A60A950792FFF71EFD4FF400437C
S3150800172C0A264FF0FF08C9F8103000F02BFE00F11E
S3150800173C640503E000F026FE854202D3A3689907E8
S3150800174CF8D584F80C8000F01DFE00F1640503E062
S3150800175C00F018FE854202D3A368DA07F8D5013ED5
S3150800176CE3D1092103224FF48058694C674B089141
S3150800177C204607A9099207930A96FFF7EDFCC4F8C9
S3150800178C148031463046FFF7B7FE012805460FD0C0
S3150800179C604BFF201E60C4F81080FFF765FE3B788F
S315080017AC43F001033B703878C0B216B0BDE8F08739
S315080017BC00F0E8FD4FF4D57100F57A780820FFF7AC
S315080017CC9BFE012818D107AC254608AEFF20FFF76B
S315080017DC4BFE05F8010BB542F8D19DF81E30012BCE
S315080017EC57D000204FF480524A49494B08601A6179
S315080017FCFF20FFF739FED2E73146A920FFF77CFE1A
S3150800180C02283ABFA9250224012406E0002128460D
S3150800181CFFF772FE28B100F09FFE00F0B3FD4045BD
S3150800182CF4D300F0AFFD4045DBD24FF40071102025
S3150800183CFFF762FE0028D4D14FF480523549344B59
S3150800184C0C60FF201A61FFF70FFE00234FF4827E0F
S3150800185C4FF4007C082607253A782B4C02F0FE023A
S3150800186C3A7022680CA922F04002226020460C939A
S3150800187CCDE90E331093CDE91333CDF834E0CDE929
S3150800188C11C61595FFF75EFD236843F040032360E8
S3150800189CE1E69DF81F30AA2BA3D105E04FF0804155
S315080018ACA920FFF729FE18B100F06CFD4045F5D3C9
S315080018BC00F068FD404594D200213A20FFF71CFE43
S315080018CC00288ED1FF20FFF7CFFD04F8010BAC42A0
S315080018DCF8D19DF81C304FF480525B064CBF0C2097
S315080018EC04200C490A4B08601A61FF20FFF7BCFD5F
S315080018FCABE700BF0C0000200010024010001004DB
S3150800190CA000A00440004004003800408000800479
S3150800191C000C01403004002018B9034B1878C0B2EB
S3150800192C70470120704700BF0C00002038B5E0B99D
S3150800193C1C46D3B1204B1B78D8072CD41F4B0D460D
S3150800194C1B681B0758BF5202012C114626D01220C1
S3150800195CFFF7D2FD80B101244FF48052184BFF20BB
S3150800196C1A61FFF781FD204638BD0424204638BD90
S3150800197C00F0F2FD013C09D028464FF40071FFF740
S3150800198C2FFE05F500750028F2D1012400210C2044
S3150800199CFFF7B2FDE0E70324204638BD1120FFF718
S315080019ACABFD0028D8D128464FF40071FFF718FE76
S315080019BCB0FA80F46409CFE70C000020300400204C
S315080019CC000C014030B583B018BB1C460BB3334B27
S315080019DC0D461978C9073DD41B7858073ED4304BA9
S315080019EC1B68190758BF5202012C42D013F0060F78
S315080019FC38D111461920FFF77FFDD8B101244FF4D1
S31508001A0C8052284BFF201A61FFF72EFD204603B0A3
S31508001A1C30BD0424204603B030BDFC20FFF724FD5E
S31508001A2C2846FFF7BDFD05F5007538B100F094FDA5
S31508001A3C013C03D0FFF732FD0028EED1FFF72EFD4F
S31508001A4C0028DBD000344FF0FD0018BF0124FFF747
S31508001A5C0BFDD4E70324204603B030BD02242046F0
S31508001A6C03B030BD214697200192FFF745FD019A38
S31508001A7CBFE711461820FFF73FFD0028BED1FFF738
S31508001A8C0DFD0028BAD0FE20FFF7EEFC2846FFF71E
S31508001A9C87FDB0FA80F46409B1E700BF0C0000209A
S31508001AAC30040020000C014070B584B0A8B9844BF2
S31508001ABC1B78D8070DD415460E2900F2AD80DFE841
S31508001ACC01F0804DAB2AABABABABABAB9E8FA31780
S31508001ADC10000324204604B070BD0424204604B02C
S31508001AEC70BD784B1B685B0700F1BB8001246DE069
S31508001AFC00213A20FFF700FD0028F7D16C1E0335AC
S31508001B0CFF20FFF7B1FC04F8010F00F025FDA542F4
S31508001B1CF6D100245AE06B4E316811F004017DD0E1
S31508001B2C00218D20FFF7E8FC0028DFD1FF20FFF706
S31508001B3C9BFC10216846FFF753FD0028D6D03024AD
S31508001B4CFF20013CFFF790FC14F0FF04F8D110239A
S31508001B5C9DF80A20120993402B6037E000210920D2
S31508001B6CFFF7CAFC04460028C0D110216846FFF7C7
S31508001B7C37FD0028BAD09DF800309B09012B00F0E0
S31508001B8C82809DF807309DF808609DF806009DF840
S31508001B9C05209DF809109B0003EB96139DF80A6027
S31508001BAC800202F00F02490000F4406002EBD612E4
S31508001BBC01F0060103440A440133073A93402B60AB
S31508001BCC04E0FFF781FCB0FA80F464094FF4805204
S31508001BDC3D4BFF201A61FFF747FC204604B070BD49
S31508001BEC00210920FFF788FC00287FF47FAF2846E0
S31508001BFC1021FFF7F5FCB0FA80F46409E6E7314BDF
S31508001C0C00241B681370E1E700210A20FFF774FC17
S31508001C1C00287FF46BAFEAE70424D7E70920FFF71F
S31508001C2C6BFC044600287FF461AF10216846FFF769
S31508001C3CD7FC00283FF45AAF32689DF80A3012F0E8
S31508001C4C02029DF80B002ED05B009DF80D2003F0C8
S31508001C5C7E0303EBD01392090133013A93402B60B0
S31508001C6CB4E700218D20FFF747FC00287FF43EAF30
S31508001C7CFF20FFF7F9FB28464021FFF7B1FCB0FA25
S31508001C8C80F46409A2E79DF807209DF80810120451
S31508001C9C9DF8093002F47C12013203EB012313443C
S31508001CAC9B022B6092E7C100C3F3840301F0180171
S31508001CBC013301EB501101FB033314462B6085E706
S31508001CCC0C00002030040020000C014072B670474E
S31508001CDC62B670472DE9F0438BB06846FFF706FBF2
S31508001CEC0298314B314AA3FB003000250224052605
S31508001CFC4FF4FA7702F1220C800902E09678D47830
S31508001D0C0232331903FB0773B0FBF3F103FB110320
S31508001D1C23B98DB26B1EB3F5806F40D39445EDD1C4
S31508001D2CB421234800F04AFB224C234E4FF00008FE
S31508001D3C4FF00109214F224B3846C7E90035C7E950
S31508001D4C046487F8188087F8198087F81A8087F84A
S31508001D5C1C8087F81D80C7E9028887F81B904CF60B
S31508001D6CE045FEF7FBFC4FF6E07404220E236946A9
S31508001D7C3846CDE902420993CDE90588CDF81C9081
S31508001D8CCDF80480CDF81080CDF820900095FEF79C
S31508001D9C67FD3846FEF7E0FD0BB0BDE8F083013E63
S31508001DAC013C36042405C1E7D34D62108C5000085B
S31508001DBC505000080000F0FF0000FFFF340400201C
S31508001DCC0064004030B540F2E175002489B00691F4
S31508001DDC024601AB02A90E480295CDE90444FEF76A
S31508001DECEBFD08B109B030BD00F0CCFA084C00F197
S31508001DFC320505E000F0B0FB00F0C4FAA842F1D8B1
S31508001E0C01992046FEF734FE0028F3D109B030BDFF
S31508001E1C3404002010B588B00C46034601AA0021EC
S31508001E2C0A48FEF735FE70B940F26763019A9A4282
S31508001E3C01D008B010BD039B002BFAD10120059BDD
S31508001E4C237008B010BD002008B010BD3404002063
S31508001E5CFFF73CBF10B500F0B9F900B910BDFEF795
S31508001E6C73F90028FAD000F041FBFEF725FC00F0C8
S31508001E7C73FA00F0ADF9074B20F0604020F07F00B4
S31508001E8C986000F0A5F94468FFF722FF2346BDE8E1
S31508001E9C1040184700ED00E072B170B5541EA4B29C
S31508001EAC0C440134461A0B784D1C8B5500F054FB28
S31508001EBCA5422946F7D170BD704700BF2DE9F843F6
S31508001ECC80460024FEF7EEFE08F1040906E0A35945
S31508001EDC0434AB4217D1B4F5007F1AD0D8F8006099
S31508001EEC59F80450A71900F037FB2A46394600233F
S31508001EFC0220FEF723FF0028E9D00024FEF7E6FEB1
S31508001F0C2046BDE8F8830446FEF7E0FE2046BDE809
S31508001F1CF8830124F2E700BF70B50F4C0D46A042BA
S31508001F2C15D00E4B99420CD123689D4207D02046FA
S31508001F3C294640F8045B4FF40072FFF7ADFF2046C4
S31508001F4C70BD0646FFF7BAFF18B13446ECE7044CE9
S31508001F5CEAE70446F3E700BF6006002000600008C5
S31508001F6C5C0400202DE9F8430C46016824F4FF783C
S31508001F7C1D464B1C0746164628F0010833D08845E3
S31508001F8C26D10434641A3C4408F5007807F1040990
S31508001F9C05E016F8013B013D04F8013B15D000F0AD
S31508001FACDBFAA4EB0903B3F5007FF2D338464146B6
S31508001FBCFFF7B2FF074600F1040988B14C4616F83C
S31508001FCC013B013D04F8013BE9D10120BDE8F8834A
S31508001FDC38464146FFF7A0FF074608B10168D0E727
S31508001FEC0020BDE8F883814649F8048B41464846EB
S31508001FFC4FF40072FFF750FF3968C0E74FF0FF3314
S3150800200C0249034A0B601360704700BF5C0400204A
S3150800201C60060020104B30B44D1E1C1AA54213D86E
S3150800202C0E4CA04210D9441E0C449C420CD820F4E9
S3150800203CFF730B4C23F00103A3420B46014606D053
S3150800204C30BC0848FFF78EBF002030BC70470648E6
S3150800205C30BCFFF787BF00BFFFFF0108FF5F000812
S3150800206C006000085C04002060060020002330B5E0
S3150800207C1F4C4D1E221A87B09542019332D820F474
S3150800208C7F721C4D22F00302AA422BD9451E0D4421
S3150800209CA54227D80D18AD1AC5F30903C5F38F2524
S315080020AC0BB10135ADB200240123049202940593B9
S315080020BCFEF7F8FD35B919E0049B954203F58063E4
S315080020CC049313D900F048FA01A902A8FEF78CFE6E
S315080020DC0134A2B20028EFD00024FEF7F7FD204603
S315080020EC07B030BD1C46204607B030BD0124F4E7C6
S315080020FCFFFF0108FF5F00080F490B68013318D072
S3150800210CD1E9013010B5CC680344086923444C69FD
S3150800211C034488692344C969034482B00B4402AA60
S3150800212C5B4242F8043D04210448FFF773FF02B0F2
S3150800213C10BD0120704700BF600600200C61000826
S3150800214C0D4A0E4B0E4910681B6810B40C680344F4
S3150800215C906823448C68034410311069234402F5B3
S3150800216C84720968034412680B44D3420CBF0120DD
S3150800217C002010BC704700BF04600008006000080F
S3150800218C086000080A4808B5036801330BD10948EA
S3150800219C0368013305D0FFF791FE003018BF012004
S315080021AC08BD012008BDFFF789FE0028EFD108BD40
S315080021BC600600205C040020004870470060000898
S315080021CCFFF71CBFFFF726BFFFF750BFFFF7B8BFD7
S315080021DCFFF7F2BF08B5FFF78FFF00B908BDBDE8DA
S315080021EC0840FFF7CFBF00BF38B5084C606000F059
S315080021FCC9F800F10A0505E000F0AEF900F0C2F8DE
S3150800220CA84202D823681B06F6D538BD0044004000
S3150800221C70B500234FF461460C250F4C88B0E26864
S3150800222C01A922F40052E2602046CDE90163CDE90A
S3150800223C0333CDE90553FFF7B7F8236923F4904325
S3150800224C2361636923F02A036361E36843F400534B
S3150800225CE36008B070BD00BF00440040402938B5A3
S3150800226C0D46044611D82846ADB2FFF7BDFF5DB141
S3150800227C013DADB22544013C00F06EF914F8010F8E
S3150800228CFFF7B2FFAC42F7D138BD6F21014800F019
S3150800229C95F8E8E7B0500008F8B51F4D2C786CB9DE
S315080022AC1E4B1A68920606D55B681D49DBB25A1E88
S315080022BC3F2A0B7027D900242046F8BD174A166802
S315080022CC16F0200615D0174C0F4623781449566875
S315080022DCCA18567001330A78DBB29A422370EAD1CF
S315080022EC0131FFF7D9FD002223782A703B700124AF
S315080022FCE2E700F047F80C4B1B6864339842DAD9CE
S3150800230C34462E70D8E700F03DF801220649054BF5
S3150800231C08602A701C70CFE7A5080020004400400E
S3150800232C64080020A6080020A80800200022052022
S3150800233C10B4064B064C07491A605A609A605C60E2
S3150800234C9A6010BC18600A60704700BF10E000E085
S3150800235C3F190100AC0800200022024B1A605A6093
S3150800236C9A60704710E000E0044B1B68DB0303D54A
S3150800237C034A136801331360704700BF10E000E08E
S3150800238CAC080020044A054B12681868D20344BFEF
S3150800239C01301860704700BF10E000E0AC08002060
S315080023AC044A054B12681868D20344BF01301860FA
S315080023BC704700BF10E000E0AC08002008B500F03C
S315080023CCCBF8FCE710B500F0BDF8012806D000F0F4
S315080023DC2FF918B10C4C2378012B00D010BDFFF740
S315080023ECD1FF0A4B0A4A1B681268134403F5FA73A1
S315080023FC9842F3D30023237000F022F90028EDD17C
S3150800240CBDE81040FFF726BDB4080020B008002030
S3150800241CB8080020012208B5044B1A70FFF7B2FF62
S3150800242C034B1860BDE80840FFF7CCBFB408002082
S3150800243CB808002008B5FFF70BFD00F08BF8FFF77E
S3150800244C75FFFFF7BDFE00F0D9F800F013F8BDE8EC
S3150800245C0840FFF7DFBF00BF08B500F07DF8FFF7AF
S3150800246C83FF00F0E7F900F015F8BDE80840FFF720
S3150800247CA9BF00BF10B500F017FCFFF72BFC012312
S3150800248C034C2370FFF7C4FE0023237010BD00BF56
S3150800249C0D00002000B583B00DF107011148FFF7B8
S315080024ACB9FC012814D00DF107010E48FFF7F4FE0C
S315080024BC012802D003B05DF804FB00220A4B9DF8F4
S315080024CC071008481A7000F00BFC03B05DF804FB03
S315080024DC0346054A9DF807100248137000F000FCE5
S315080024ECE1E700BFBC0800200D000020704700BFC4
S315080024FC70B50A4C0D4623780646012B08D01BB935
S3150800250CE9B23046FFF7AAFEBDE8704000F0E0BB22
S3150800251CC9B2FFF757FC2378F1E700BF0D0000207E
S3150800252C054B1B78013BDBB2022B9ABF034A32F8E8
S3150800253C13004020704700BF0D000020F050000823
S3150800254CFFF7EEBF08B500F0BBFB003018BF012043
S3150800255C08BD00BFFDF706BEFDF708BE092802D95F
S3150800256C3730C0B2704710B500F13003DCB202F058
S3150800257C03FD23462044427802F00302022A08BFD0
S3150800258CA4F12003D8B210BD38B5054600090C468F
S3150800259CFFF7E4FF207005F00F00FFF7DFFF0023BD
S315080025AC6070A370204638BDF8B50027461E451C3A
S315080025BC16F8014F02F0E0FC23462044417801F05E
S315080025CC0301022908BFA4F12003DBB2A3F13002F0
S315080025DCD2B2162AA3F13A010DD806290BD9092A23
S315080025EC84BF373BDAB202EB0713AE4203F0FF07A0
S315080025FCDED13846F8BD00273846F8BD002310B59D
S3150800260C074C1A4607490848237001F065FF00B9BC
S3150800261C10BD7721BDE810400448FFF7CFBE00BFB8
S3150800262C5C0D0020F850000804090020FC50000836
S3150800263C024B1878B0FA80F0400970475C0D002000
S3150800264C10B5FFF77FFF012802D0054C23780BB194
S3150800265C002010BDFDF78CFD0128F9D1207010BDA6
S3150800266C5C0D002038B50546047802F085FC234637
S3150800267C2044427802F00302022A08BFA4F1200380
S3150800268C532B01D0032038BD02F076FC6B78184426
S3150800269C42785207F6D5312B05D0322B05D0332B81
S315080026ACF0D1022038BD002038BD012038BD00BF4E
S315080026BC70B506460230FFF777FF0546043684B236
S315080026CC3046FFF771FF013CA4B20544012CEDB26C
S315080026DC06F10206F4D83046ED43FFF765FFEDB276
S315080026EC281AB0FA80F0400970BD00BFF8B5044648
S315080026FC16460D46002946D0002844D02046FFF73A
S3150800270CB1FF032807463BD02046FFF7D1FF002828
S3150800271C00F08B80012F3CD065D3022F30D1A01C42
S3150800272CFFF742FF0746201DFFF73EFF000628600D
S3150800273CA01DFFF739FF2B68053F03EB0040286007
S3150800274C04F10800FFF730FF2B683FB203EB0020BB
S3150800275C286004F10A00FFF727FF2B6803442B6057
S3150800276C7EB1002F0DDD00250C342046FFF71CFF2B
S3150800277C6B1C70559DB2BD4204F10204F5DB00E0FA
S3150800278C00273846F8BD40F263212948FFF716FEA4
S3150800279CB4E7A01CFFF708FF0746201DFFF704FF48
S315080027AC00042860A01DFFF7FFFE2B68043F03EB0F
S315080027BC0020286004F10800FFF7F6FE2B683FB2EC
S315080027CC03442B60002EDCD0002FDADD00250A34FA
S315080027DC2046FFF7E9FE6B1C70559DB2BD4204F10D
S315080027EC0204F5DBCDE7A01CFFF7DEFE0746201D2D
S315080027FCFFF7DAFE00022860A01DFFF7D5FE2B684E
S3150800280C033F03443FB22B60002EBAD0002FB8DD2D
S3150800281C002508342046FFF7C7FE6B1C70559DB281
S3150800282CBD4204F10204F5DBABE74FF0FF37A8E72E
S3150800283CFC5000082DE9F843C14D2C782CB1012C1D
S3150800284C05D0022C64D0032C20D0BDE8F883FFF702
S3150800285CB7FCFDF7AFFCBB48FDF7ECFCBA48FDF737
S3150800286CE9FCFDF7A3FC22460146B84801F062FED6
S3150800287C0646002800F0CB800023B5482B70FDF7E0
S3150800288CD9FC2046BDE8F843FDF7CABCB14EB24F99
S3150800289C06F50C7238464FF4807102F083FA96F8F6
S315080028AC4192B9F1000F40F0CF8070B107F58072F4
S315080028BC07F5C0713846FFF719FFB0F1FF3F8046A0
S315080028CC00F02181002800F3C280D6F84422D6F8FD
S315080028DC3C329A42B9D1A148FDF7ACFCFFF77AFC19
S315080028EC0346002800F01F819D48FDF7A3FC9D4870
S315080028FCFDF7A0FC954802F009F99B48FDF79AFCF0
S3150800290C00232B70FDF76AFCBDE8F843FFF7A2BA63
S3150800291C904E914F06F50C7238464FF4807102F0C2
S3150800292C41FA96F84182B8F1000F7FD1A8B1424618
S3150800293C07F5C0713846FFF7D9FEB0F1FF3F81465F
S3150800294C00F0D380002808DD884CD7F8802163680E
S3150800295C002B40F0C380C4E90020D6F84422D6F8F0
S3150800296C3C329A427FF471AF0021784802F0E0F8C5
S3150800297C002840F067817D4C6368002B41D078486D
S3150800298CFDF758FC7A48FDF755FC636879491A46F1
S3150800299C7948A0FB0262D20801F10101F9D1764E01
S315080029AC0A70A6FB0302D20802EB8200A3EB4003D3
S315080029BC303301F8013D1346002AF2D16D48FDF774
S315080029CC39FC6E48FDF736FC6A49E078FFF7DCFD02
S315080029DC6B49A078FFF7D8FD6A496078FFF7D4FDF4
S315080029EC69492078FFF7D0FD6248FDF723FC674854
S315080029FCFDF720FCD4E90001FFF7E6FB002800F000
S31508002A0C2E815748FDF716FC03232B701DE75448F7
S31508002A1CFDF710FC5E48FDF70DFC5E48FDF70AFC59
S31508002A2C0222524B2A70C3E900660EE70023484877
S31508002A3C2B70FDF7FFFB0220FDF7F2FB06F50C7079
S31508002A4CBDE8F84302F062B800235348F0E7534850
S31508002A5CFDF7F0FB43464749474AA2FB0303DB084D
S31508002A6C01F10101F9D1444643480B70A0FB04233C
S31508002A7CDB0803EB8302A4EB4202303201F8012D8A
S31508002A8C1C46002BF2D13B48FDF7D4FB4448FDF716
S31508002A9CD1FB384997F88301FFF776FD384997F843
S31508002AAC8201FFF771FD374997F88101FFF76CFD35
S31508002ABC354997F88001FFF767FD2E48FDF7BAFBF5
S31508002ACC3248FDF7B7FB4146D7F88001354AFFF780
S31508002ADC79FBE0B12248FDF7ADFBF6E6216819440F
S31508002AEC914263D10344636037E7194885F800803F
S31508002AFCFDF7A0FB0320FDF793FB06F50C70BDE86C
S31508002B0CF84302F003B8284885F80090F0E7104817
S31508002B1C2C70FDF78FFB0620FDF782FBBDE8F8430A
S31508002B2C0A4801F0F3BF0A482B70FDF783FB072010
S31508002B3CFDF776FBBDE8F843044801F0E7BF00BF94
S31508002B4C5C0D00202C51000850510008340B002055
S31508002B5C7851000804090020600D00207452000802
S31508002B6C8051000890520008A8520008FC08002062
S31508002B7CDC510008E40E0020CDCCCCCCE851000882
S31508002B8CE60E0020E80E0020EA0E00208C52000803
S31508002B9C88510008AC510008045200084C52000831
S31508002BAC5C520008600E0020285200083248FDF7D7
S31508002BBC41FB3248FDF73EFB636831491A463148FA
S31508002BCCA0FB02C2D20801F10101F9D1DFF8B4C0A9
S31508002BDC0A70ACFB0302D20802EB8200A3EB40039B
S31508002BEC303301F8013D1346002AF2D12448FDF78B
S31508002BFC21FB2548FDF71EFB2149E078FFF7C4FCAD
S31508002C0C2249A078FFF7C0FC21496078FFF7BCFC85
S31508002C1C20492078FFF7B8FC1948FDF70BFB1E482E
S31508002C2CFDF708FBD4E90001FFF7CEFAB8B1124854
S31508002C3CFDF700FB1948FDF7FDFAD7F88031C4E912
S31508002C4C00398AE6002316482B70FDF7F3FA0420A0
S31508002C5CFDF7E6FABDE8F843124801F057BF002322
S31508002C6C0F482B70FDF7E6FA0520FDF7D9FABDE8F3
S31508002C7CF8430C4801F04ABF80510008DC510008A3
S31508002C8CE40E0020CDCCCCCCE8510008E60E002092
S31508002C9CE80E0020EA0E00208C520008AC51000801
S31508002CAC78510008340B00200022044B9A6483F8F0
S31508002CBC4320A3F844201A809A707047240F0020EA
S31508002CCC024B1878003018BF01207047240F0020DB
S31508002CDC0022024B83F84320704700BF240F0020C4
S31508002CECF8B50578FF2D41D0B04C2378012B00D0D0
S31508002CFCF8BDC93D0646352D00F23C81DFE815F0D6
S31508002D0C23013A013A018D003A013A0105017A008C
S31508002D1C0D0114013A013A013A013A013A013A0114
S31508002D2C3A013A013A013A013A013A013A013A01B1
S31508002D3C3A013A013A013A013A013A013A013A01A1
S31508002D4C3A013A013A013A013A013A013A013A0191
S31508002D5C3A013A019500B000BE00D2003A013A0198
S31508002D6C3A01DA003A01E900F100FD00FFF760FCD0
S31508002D7CA8B9FE21102202238C4CE1702271A4F80A
S31508002D8C443094F84330012B2CD0B4F8441001236A
S31508002D9C874884F84330BDE8F840FFF7A9BB002301
S31508002DAC10220126814C637122712680E570FFF78B
S31508002DBCB7FBA071FFF7C4FBE071FFF7C1FB082353
S31508002DCCD84020726672A672A4F84430FFF7F8F958
S31508002DDC94F84330012B05D0B4F94410002987DD4B
S31508002DEC89B2D4E7FE2210230221E2702371A4F8DB
S31508002DFC4410CCE7FFF794FB73780138984235DD1D
S31508002E0CFF220123E270A4F844307178002940F0BF
S31508002E1CBE80FFF7DFF90028DAD1FE213122022322
S31508002E2CE1702271A4F84430ABE7FF23E3704768DE
S31508002E3CA66C002F00F0B7800025374416F8013B26
S31508002E4C1D44FFF789FBB742EDB2F7D101210022E9
S31508002E5C0823C4F80750A180A271A4F8443090E75F
S31508002E6CFFF75EFB73788342C0F08C80FE2122222A
S31508002E7C0223E1702271A4F8443082E7FFF750FB75
S31508002E8C72789042F2D9A16C4A48FFF705F8FF23ED
S31508002E9CE3707278A36C1344A36473780133A4F8B3
S31508002EAC443095E7FF230122E3704368A4F84420D5
S31508002EBCA36466E70023FF25072008213E4AE57030
S31508002ECC23716371A371C4F80700A4F84410A264B3
S31508002EDC57E7FE2100220223E1702271A4F8443040
S31508002EEC4FE70023FF2006216278E0702371E38008
S31508002EFC2372A4F84410627143E70021FF220123D0
S31508002F0C2180E270A4F844303BE7FEF7A3FFFF22CA
S31508002F1C0123E270A4F8443033E74168A06CFFF74C
S31508002F2C53F90028F3D178E70025FF232571E370C0
S31508002F3C6571FFF7F5FA0723A071E57125726572BD
S31508002F4CA4F844301DE7A56CFFF7EAFA721C411E7B
S31508002F5C2846FFF737F900283FF45FAFFF23E370E5
S31508002F6CFFF7DEFA0122A36C01380344A364A4F824
S31508002F7C442006E7FE2120220223E1702271A4F8E0
S31508002F8C4430FEE671680B48A16472787DE7B21C82
S31508002F9CA06CFFF717F900283FF43FAF7278A36CC3
S31508002FAC1344A36414E73D4650E700BF240F0020E2
S31508002FBC270F0020280F0020D452000830B40468CC
S31508002FCCECB125781F2D0AD93A2D18D0234602E0E4
S31508002FDC3A2A08D00B465A78591C1F2AF8D80022C8
S31508002FEC30BC104670470134A142A5F1300206D117
S31508002FFC302D04D130BC02330360104670474FF0B5
S3150800300CFF3230BC10467047D8B110B5036882B091
S3150800301C04462BB11A781AB1D888A288904204D0E3
S3150800302C002309200B6002B010BD58780191FEF7F9
S3150800303C73FC10F001000199F2D123680B6002B001
S3150800304C10BD002309200B60704700BF01380A44E5
S3150800305C11F8013B914200F8013FF9D1704700BFC6
S3150800306CF8B5C56A00F1300704462A463946407851
S3150800307C0123FEF7A7FCB0B9226AA369AA1A9A42D9
S3150800308CE0700ED2A678012E01D80AE0A3691D4479
S3150800309C013E2A46012339466078FEF793FC012E39
S315080030ACF4D10020F8BD0120F8BD00BF2DE9F84386
S315080030BCC378054663B92B78032B10D000226878A1
S315080030CC1146FEF7F1FC003018BF0120BDE8F88365
S315080030DCFFF7C6FF0028F9D12B78032BEED12B79F5
S315080030EC012BEBD105F130010B46002405F50C72CA
S315080030FC03F8014B9A42FBD14FF0520C72204FF059
S3150800310CAA0E612741264FF055082B6985F814023B
S3150800311C1A0A85F8183285F819224FEA13491A0E35
S3150800312CEB6885F81B221A0A85F81C3285F81D22CD
S3150800313C1A0C1B0E85F81F32EB6985F81E225A1CD1
S3150800314C85F8150285F81A9285F82E82EA6285F8B2
S3150800315C2FE285F830C085F831C085F8327085F8CD
S3150800316C177285F8336085F8166201236878FEF7BE
S3150800317C29FC2C71A2E700BF38B5C37804460D4666
S3150800318C13B1FFF76DFF68B92A46012304F1300124
S3150800319C6078FEF7CBFB002816BF4FF0FF350020F2
S315080031AC0120E56238BD00BF4FF0FF33002299427B
S315080031BC10B50446C270C3622BD14AF6552294F850
S315080031CC2F1294F82E3243EA012393421FD1B4F8F6
S315080031DC681094F8672094F8663042EA012243EAAC
S315080031EC0223104A23F07F43934218D0B4F8841074
S315080031FC94F8833094F8820043EA012340EA0320CA
S3150800320C20F07F40904214BF0220002010BD0320FE
S3150800321C10BDFFF7B1FF0028CFD0042010BD002049
S3150800322C10BD00BF4641540000232DE9F0410B6048
S3150800323C84B00F461546FFF7C1FE061EC0F2DC80A9
S3150800324CC24B53F82640002C00F003813C602378CF
S3150800325C05F0FE057BB16078FEF75EFBC7070AD45E
S3150800326C002D00F0038110F0040000F0C6800A203F
S3150800327C04B0BDE8F0810023F0B260702370FEF74D
S3150800328CE1F9C60700F1BC800DB14507EFD4002162
S3150800329C2046FFF789FF022800F0B680042800F0C4
S315080032ACE380012800F2D180002694F83C2094F89B
S315080032BC3B3043EA0223B3F5007F40F0C68094F80E
S315080032CC472094F8463053EA022309D1B4F856102D
S315080032DC94F8553094F8542043EA012342EA032320
S315080032EC94F84020A361511E0129A27000F2AD800A
S315080032FC94F83D1088B26081002800F0A680481E1C
S3150800330C084240F0A28094F8420094F8415045EAED
S3150800331C00252807258140F0988094F8447094F885
S3150800332C430050EA072009D1B4F852C094F85170FA
S3150800333C94F8500047EA0C2740EA072094F83FC057
S3150800334C94F83E7057EA0C2C7FD003FB02F20CEB78
S3150800335C15171744B84278D3C01BB0FBF1F10029F6
S3150800336C73D040F6F57E4FF6F57871458CBF4FF065
S3150800337C020E4FF0010E41450CEB0600374401F1E5
S3150800338C020C75D994F85B1094F85A20C4F814C03A
S3150800339C52EA0122C4E90760A76256D1002D54D11E
S315080033ACB4F85E5094F85D0094F85C104FEA8C0201
S315080033BC40EA052002F2FF1241EA0021B3EB522F34
S315080033CC616242D34FF0FF32802194F8610094F881
S315080033DC6030226143EA0023012BE26021716AD036
S315080033EC4FF0030E5A4A84F800E013880020013384
S315080033FC9BB21380E38000E00B2004B0BDE8F0819B
S3150800340C032004B0BDE8F0816D46294604F5FC732B
S3150800341C04F50E7613F8062C42B11F8813F8010C26
S3150800342C13F8022C40EA072042EA00221033B34272
S3150800343C41F8042BEED105F1100755F8046B66B963
S3150800344C0320AF42F9D104280ED00D2004B0BDE8F4
S3150800345CF0810C2004B0BDE8F08131462046FFF718
S3150800346CA3FE0128EDD820E70120C6E72846C4E7C5
S3150800347CC4F814C0C4E90760A762002DE5D002445D
S3150800348CBEF1020F626213D04FF0010E0CEB4C0228
S3150800349C0CF0010C0CEB520C0CF2FF1CB3EB5C2F72
S315080034ACD3D34FF0FF338022C4E90333227199E753
S315080034BC4FEA4C0CF0E7E36A711C994204D020469B
S315080034CCFFF75AFE00288BD14AF65522002094F8AD
S315080034DC2F1294F82E32207143EA012393427FF47B
S315080034EC7FAF618E94F8312094F8303042EA01228D
S315080034FC184943EA02238B427FF472AFB4F81612CA
S3150800350C94F8152294F8143242EA0122124943EA35
S3150800351C02238B427FF464AF94F8192294F81D3277
S3150800352CB4F81A02B4F81E1242EA002043EA012142
S3150800353C94F8182294F81C3242EA002243EA012332
S3150800354C4FF0030EC4E903324CE700BF700F00209E
S3150800355C740F0020525261417272416101292CD9B3
S3150800356C4269F8B59142074625D202780C46022ADA
S3150800357C3DD0032A23D0012A1DD1036A01EB51063B
S3150800358CD0F82CC003EB562161454CD1C6F3080282
S3150800359C013603EB56213A44614592F830504AD12C
S315080035ACC6F30806BB1993F83000E30745EA002072
S315080035BC47D50009F8BD0120F8BD01207047016AFE
S315080035CCC36A01EBD411994228D1A10001F4FE710A
S315080035DC01F130033B445A8839445B7891F8300042
S315080035EC43EA022340EA032020F07040F8BD016A42
S315080035FCC36A01EB1421994205D0FFF7BDFD10B142
S3150800360C4FF0FF30F8BD610001F4FF71394491F8B1
S3150800361C313091F8300040EA0320F8BDFFF7ACFDD5
S3150800362C0028D2D0ECE7FFF7A7FD0028E8D13B6AC3
S3150800363CD7F82CC0AAE73846FFF79EFD0028AFD06E
S3150800364CDEE7C0F30B00F8BDB1F5001F29D2CA0698
S3150800365CF8B50C4623D1816805460461066819BB82
S3150800366C3378022B01D9736AEBB93389B3EB541F40
S3150800367C15D9736AAB6169618BB1C4F3080230362C
S3150800368C03EB54241644C5E906460020F8BD7369B5
S3150800369C023B8A1E9A421ED30023C5E90513022053
S315080036ACF8BD02207047194677897F02BC42EED3D3
S315080036BC304607E00128F2D973698342EFD9A7424D
S315080036CCE6D82868FFF74AFF431C0146A4EB070413
S315080036DCF0D10120F8BD7389B06A02FB0303AB6114
S315080036ECC9E700BF2DE9F04103780446022B0D46C5
S315080036FC164655D0032B32D0012B02D00220BDE83A
S3150800370CF081036A01EB5107C26A03EB5721914218
S3150800371C5FD107F1010803EB5821EB07C7F308073C
S3150800372C63D50120274497F830308A4203F00F03FB
S3150800373C43EA061387F83030E07004D02046FFF7CA
S3150800374C1BFD0028DBD1C8F30808C6F30716A044EE
S3150800375C012388F83060E3700020BDE8F081016A27
S3150800376CC36A01EBD51199423AD10127AD0005F48C
S3150800377CFE7505F1300121444B8826F070461A0473
S3150800378C02F070423243254485F83020100A130C97
S3150800379C120E48708B70CA70E7700020BDE8F08175
S315080037AC016AC36A01EB1521994203D0FFF7E4FCC1
S315080037BC0028A4D101239D4005F4FF752544C6F3C2
S315080037CC072285F8306085F83120E3700020BDE8C3
S315080037DCF081FFF7D1FC002891D1236AE26A98E7B9
S315080037ECFFF7CAFC0028C0D089E7012327448A4280
S315080037FC87F83060E3700AD1C8F30808A04498F833
S3150800380C3030C6F3032223F00F061643A0E72046F2
S3150800381CFFF7B2FC00287FF472AFEDE72DE9F04113
S3150800382C07468846066829BBF5687369F5B9012504
S3150800383C2C4606E0012815D0013031D0AC4234D0E4
S3150800384C736901349C4202D3012D2ED902242146D8
S3150800385C3868FFF783FE0028ECD1012C02D973696E
S3150800386C9C4214D301242046BDE8F0819D4228BF12
S3150800387C0125DDE73046FFF771FE01280446F1D92C
S3150800388C431C0DD073698342EDD84546D0E74FF0FB
S3150800389CFF3221463046FFF725FF50B10128E1D10A
S315080038AC4FF0FF342046BDE8F08100242046BDE8E1
S315080038BCF081B8F1000F0CD0B8F1010FD2D97369A9
S315080038CC9845CFD2414622463046FFF70BFF0028D3
S315080038DCE4D1D6E90423023B9A42F46001D2013AB8
S315080038EC3261337943F001033371BCE72DE9F84FA4
S315080038FC8369CBB105692035B5F5001F14D2C5F31C
S3150800390C08068846044607683EB94169013383614F
S3150800391C69B93B89B3EB551F29D930363E44E66164
S3150800392C25610020BDE8F88F0420BDE8F88F7B8957
S3150800393C013B13EA5523F0D13846FFF70FFE012851
S3150800394C81465CD9B0F1FF3F19D07B69834218D9FF
S3150800395CA0F10208023B434592BF00237B89BA6A51
S3150800396CC4F8149088BF08FB0323A361D5E700238A
S3150800397C0420A361D9E73846FFF772FB98B10120FA
S3150800398CD3E7B8F1000FF2D061692046FFF746FF7E
S3150800399C8146002835D0012831D0B0F1FF3FEED052
S315080039ACFB78002BE7D1002207F1300307F50C71E1
S315080039BC03F8012B9942FBD17B69A9F102089A1EDF
S315080039CC90452CBF0022BA6A798938BF08FB0122B8
S315080039DCFA62E9B14FF0000B4FF0010A05E0FA6AFA
S315080039EC7B8901325B45FA620DD987F803A0384604
S315080039FCFFF736FB0BF1010B0028F0D0BFE70220CE
S31508003A0C93E7072091E77B69A2EB0B02FA62A1E721
S31508003A1C8B46F9E7416A2DE9F0414B1C04460568CB
S31508003A2C06691AD14FF0E508012704E00021204663
S31508003A3CFFF75CFFB8B9A169EB6A994203D028462F
S31508003A4CFFF79AFB78B9E36983F80080EF7023696E
S31508003A5CB342EBD30020BDE8F081FFF7F5FD002853
S31508003A6CE0D0BDE8F081042808BF0220BDE8F0814B
S31508003A7C2DE9F04F002187B005460768FFF7E4FDEE
S31508003A8C8246002847D14FF0FF334FF0FF0B98467C
S31508003A9CD9466B620CE00F2B41D04FF0FF09C5F8E5
S31508003AAC248000212846FFF721FF002840F0A38038
S31508003ABCA969FB6A994205D03846FFF75DFB0028D1
S31508003ACC40F09980EC692678002E00F09980E27A0D
S31508003ADCE52E02F03F03AB71DFD01207DBD40F2BB8
S31508003AEC1DD0B9F1000F6AD0296ACB7ADB07D4D47A
S31508003AFC0846237810F80B2B01319B1A0134002B3E
S31508003B0CCBD111F8012B14F8013B8842A3EB020325
S31508003B1CF5D1002BC1D1504607B0BDE8F08FAB6A82
S31508003B2C002BBED070065BD52A6994F80DB006F04A
S31508003B3CBF066A62627B5A4554D1E17EA27E52EA7E
S31508003B4C01224FD101212278CDE901B702F03F02BB
S31508003B5C013A02EB420002EB8002CDE903A5059679
S31508003B6C254693461C46DFF8D8900B4613E0BBF166
S31508003B7CFE0F1DD8304601F085F9824634F81B0035
S31508003B8C01F080F9824513D13346BB462B4A4A4588
S31508003B9C3CD019F8011F681840786E5C0BF10107C8
S31508003BAC46EA0026002BE2D14FF6FF729642EDD07C
S31508003BBCDDE901B7DDE903A54FF0FF0971E72146F9
S31508003BCC04F10B0011F8012B4FEAC91343EA590902
S31508003BDC9144884209F0FF09F4D1CB4584D19AE780
S31508003BECB145A7D0002128464FF0FF09FFF77EFE06
S31508003BFC00283FF45DAF8246504607B0BDE8F08F0B
S31508003C0C4FF0040A504607B0BDE8F08F9C46234691
S31508003C1C2C46DDE903A521785A464906029F059EDE
S31508003C2CDDF804B006D5BCF1000F03D033F812301A
S31508003C3C002BD7D1013E5FFA86F932E768530008A4
S31508003C4C5C5300082DE9F04FD0F820A08BB09AF8F9
S31508003C5C0B3013F0A00840F0F180D0F82890B9F892
S31508003C6C0030002B00F07E814B4633F8022F08F10A
S31508003C7C0108002AF9D10446236807A80C225146E4
S31508003C8C0093FFF7E3F99DF82730DD0755D49B071A
S31508003C9C40F1D180B44B08F10C08A3FB08384FEA65
S31508003CAC980808F10108002120462768FFF7CCFC84
S31508003CBC0546002840F0A980064608E0ABB1002668
S31508003CCC01212046FFF712FE002840F09D80A169CD
S31508003CDCFB6A994205D03846FFF74EFA002840F0A1
S31508003CEC9380E3691B78E52BE8D10136B045E7D11B
S31508003CFCB8F10103019340F0B180009BA169DB6A1E
S31508003D0C994240F0A0800021E36903F1200203F8F0
S31508003D1C011B9342FBD10B22D4E90701FFF796F955
S31508003D2CD4E907130122DB7A03F018030B73009B03
S31508003D3CDA7028460BB0BDE8F08F002301278AF805
S31508003D4C0B300B22A36207A95046FFF77FF93B46B7
S31508003D5C864E07220DF11B0503F00F0000F130010A
S31508003D6C392988BF00F137011B0902F1FF3205F822
S31508003D7C0119F1D17E200AA9114401F8140C002A64
S31508003D8C4AD09AF80010202908D0514603E011F8B9
S31508003D9C010F202802D001339A42F8D1591E5144FA
S31508003DAC072A0AA810448CBF202010F8140C03F11B
S31508003DBC010398BF0132072B01F8010FF0D92046F1
S31508003DCCFFF756FE054648BB0137642F1FD00B225A
S31508003DDC07A95046FFF73AF9052F13D93B46A9F11F
S31508003DEC020535F8022F002AB3D0102102F0010083
S31508003DFC00EB4303D80348BF734001394FEA52021C
S31508003E0CF4D1EEE73B46A4E70546042D91D10725E8
S31508003E1C28460BB0BDE8F08F1346BFE7042888D1B7
S31508003E2C9DF827308AF80B309DF82730C4F828906F
S31508003E3C9B073FF52FAF4FF0010834E706252846B8
S31508003E4C0BB0BDE8F08F0098FFF796F900283FF401
S31508003E5C5AAF054628460BB0BDE8F08F2169019B81
S31508003E6C2046A1EB4311FFF7EFFB0028F1D1216A9D
S31508003E7C024601F10B00D30111F8016B43EA520318
S31508003E8C3344814203F0FF02F5D1DFF8E4B0029225
S31508003E9C0395009BA169DB6A994204D00098FFF749
S31508003EAC6BF90028D5D1E169029F0026D4F8288041
S31508003EBC4F734FF00F079DF804A033460AF1FF32F3
S31508003ECC02EB420002EB8002012530460E73CF72DC
S31508003EDC8E76CE764FF6FF794FF0FF0E18E038F84F
S31508003EEC123001324FEA132C4B5587F801C0BBBB75
S31508003EFC0C2E21D84FF6FF731BF80650023001F82A
S31508003F0C05E00D4485F801E00C280ED81BF8005086
S31508003F1C4B4501EB050700F10106E0D130460C28AC
S31508003F2C01F805E087F801E0F0D94FF6FF708342F7
S31508003F3C02D038F812300BB94AF0400A0123009A1D
S31508003F4C81F800A020460021D370FFF7CFFC00288B
S31508003F5C7FF47FAF019B013B01939AD1039DCCE67D
S31508003F6C3046D1E7984686E64FECC44E2110010040
S31508003F7C5C53000801293DD9F8B504680D466369F8
S31508003F8C07468B422BD932BB20461CE0012826D08B
S31508003F9C411C31D0012D22D963699D421FD2294675
S31508003FAC00222046FFF79EFBA0B923695A1C05D0B0
S31508003FBC2279013342F00102236122716369B3420B
S31508003FCC07D9354638682946FFF7C8FA0646002841
S31508003FDCDCD10020F8BD012A01D9934201D8022070
S31508003FECF8BD114620464FF0FF32FFF77BFB002841
S31508003FFCE8D0F8BD022070470120F8BD2DE9F04F36
S3150800400C0746D0F800B083B00D4611F8013B2F2BAC
S3150800401CFAD05C2BF8D00021B96028781F2840F21A
S3150800402C198180B21F28BE6A2CD92F282AD05C2861
S3150800403C28D0A6F10209A84601240EE029F8020F99
S3150800404C18F8010F631C1F281ED92F281CD05C28B2
S3150800405C1AD0B3F5807F11D01C46012100F0EEFE74
S3150800406C60B17F28EAD8222808D02A238D4A03E093
S3150800407C12F8013F002BE1D09842F9D1062003B083
S3150800408CBDE8F08F012300242B441A781D462F2AED
S3150800409C03F10103F9D05C2AF7D01F288CBF4FF027
S315080040AC00094FF004094CB106EB440232F8023D04
S315080040BC202B01D02E2B07D1013CF7D1002306204B
S315080040CC338003B0BDE8F08F002220213B6A26F826
S315080040DC142003F10B0006EB440203F8011B834280
S315080040ECFBD1B31E4FF0000801E008F1010833F8C4
S315080040FC020F2028F9D02E28F7D0B8F1000F01D0DE
S3150800410C49F00309134633F8022D2E2A01D0013C37
S3150800411CF9D1002308229A4608F1010838B3202859
S3150800412C6CD02E286FD0934219D2A0456DD07F281B
S3150800413C78D82B2800F087802C21DFF870C18142B3
S3150800414C00F081801CF8011F0029F8D1A0F141016B
S3150800415C192900F288804AF0020AC0B276E00B2AC6
S3150800416C00F09580A04552D049F003094FD93B6A17
S3150800417C1978E52902D1052119703B6A082A04BF6A
S3150800418C4FEA8A0A5FFA8AFA0AF00C020C2A46D017
S3150800419C0AF0030ABAF1030F41D019F0020F08D13D
S315080041ACBAF1010F08BF49F01009042A08BF49F0F3
S315080041BC080983F80B903846FFF75AFC3B6ADB7AFA
S315080041CC00285AD15A073FF55AAFBB79DB065CD59E
S315080041DC3B699BF80010C3F3080330335B44D87E65
S315080041EC9A7E032942EA002205D1597D1B7D43EAB2
S315080041FC012342EA0342BA60287812E749F0030918
S3150800420C36F8180088E7A045F8D10B2A3FD04FEAB4
S3150800421C8A0A5FFA8AFAA0460B220823F0E749F0C5
S3150800422C0209C6E70021CDE9003200F007FEDDE9F8
S3150800423C003249F0020930B11B49084410F8800CC9
S3150800424C00287FF476AF5F2049F00309396AC85411
S3150800425C0133D5E7802238463B6ADA7203B0BDE8EB
S3150800426CF04FFFF7F1B9A0F16101192997BF203872
S3150800427CC0B2C0B24AF0010AE8E704287FF4FFAEE0
S3150800428C13F0040F08BF0520F9E60520F7E63B6A8C
S3150800429C49F003091A78E52A7FF476AF05221A70D5
S315080042AC3B6A71E76D530008DC5200087953000825
S315080042BC2DE9F843436A814601330E461ED0876AB8
S315080042CC3888BD1CB0B16FF0130807F50077A8EB5A
S315080042DC010801F1150406E0BD420BD004F8010FE4
S315080042EC35F8020B38B1002100F0A8FD08EB0403E1
S315080042FC0028F1D10023002233449A75D9F81C40C2
S3150800430C002122464FF02E0896F816C004F10B072A
S3150800431C12F8013B202B1DD0052BA2EB040508BF78
S3150800432CE523092D3AD070184372BCF1000F10D151
S3150800433CA3F1410EBEF1190F0AD8092D34BF082571
S3150800434C102594F80CE01EEA050F1CBF2033DBB2CF
S3150800435C837501319742DBD17018BCF1000F05D17A
S3150800436C80F816C0237B002B08BF30460023437207
S3150800437CE37A3372E18B627F237F42EA012243EAB6
S3150800438C02233360627E237E43EA0223B380E27DF6
S3150800439CA37D43EA0223F380BDE8F8837018BCF1C9
S315080043AC000F01D180F8168080F809800131BAE730
S315080043BC2DE9F84FFF27044605683E46042006E01B
S315080043CCFF2600212046FFF791FA002858D1A1694B
S315080043DC002959D0EB6A8B4204D02846FEF7CCFE4E
S315080043EC00284DD1E1690A78002A48D0CB7AE52A0B
S315080043FC03F03F03A371E3D02E2AE1D023F020006B
S3150800440C0828DDD00F2B44D1500635D523694F7BB0
S3150800441C02F0BF0663624B7BBB42D1D1CA7E8B7E50
S3150800442C53EA0223CCD101220878DFF8A8C000F0A1
S3150800443C3F00013800EB40034FF6FF7A9646D4F856
S3150800444C289000EB83000CF10C0809E0FE28B7D87D
S3150800445C9E4629F810300130E0452ED01CF8012F65
S3150800446C8B1893F801B08B5C43EA0B23BEF1000F53
S3150800447CECD15345F0D0A3E7B242A1D1CBE7042047
S3150800448C0023A361BDE8F88F0028F9D10020BDE808
S3150800449CF88F6EB901F10B0011F8012BF30143EA01
S315080044AC56061644814206F0FF06F5D1BE42EDD0FB
S315080044BC4FF0FF3300206362E4E70B785B0605D503
S315080044CCFE283FF67DAF002329F81030013EF6B2E0
S315080044DC77E700BF5C53000810B584B004AB43F80B
S315080044EC041D0190184614460091FEF767FD021E3E
S315080044FC14DB0F4951F822300BB100201870019BC0
S3150800450C3BB10020012C187041F8223009D004B0B8
S3150800451C10BD184641F8223004B010BD0B2004B06B
S3150800452C10BD024601A96846FEF77EFE04B010BD12
S3150800453C700F00202DE9F04192B0019170B3002361
S3150800454C02F01F0703600446154603A93A4601A85C
S3150800455CFEF76AFE064618B1304612B0BDE8F08181
S3150800456C0399654A04AB079107A801990F93119211
S3150800457CFFF744FD05F01C03A8B90F9A92F90B2016
S3150800458C002AC0F2A1809DF82220A3B112F0110FC7
S3150800459C17D16B0740F19A800826DDE709263046C5
S315080045AC12B0BDE8F0810BB104280ED00646304691
S315080045BC12B0BDE8F081D30605D4A8077CD5D1077F
S315080045CC7AD50726C8E70426C6E707A8FFF73AFBF5
S315080045DC47F008070028E9D10E9BDDF80CC000222D
S315080045EC48216120202559749A73DA7318740E9B26
S315080045FC59769A75DA7518760E9BDD720E9B9CF8B1
S3150800460C0020D97E9D7E032A45EA012505D1597DD0
S3150800461C1A7D42EA012245EA024500229A76DA76A2
S3150800462C9CF80010032901D11A755A75002201212C
S3150800463C0E9B1A775A779A77DA778CF80310002D2F
S3150800464C57D007A82946DCF82C80FFF793FC0028DE
S3150800465CACD1DDF80CC0013DDCF82C3098453DD1C9
S3150800466CCCF80C500E9B47F02007C4E908839CF83D
S3150800467C0010D87E9A7E032942EA002205D1587D7D
S3150800468C197D41EA002142EA01420021A260D88B39
S3150800469C5A7F1B7F2774617442EA0022BCF8060015
S315080046AC43EA0223A0803046E360C4F800C0616187
S315080046BCE16112B0BDE8F081DDF80CC02A070E9B4B
S315080046CCDCF82C80D1D5CEE7062645E72D070E9BC0
S315080046DCDDF80CC083D4DCF82C80C6E7604641466E
S315080046ECFEF74AFDDDF80CC0CCF80C5000287FF418
S315080046FC5DAFDCF82C80B5E7780F00202DE9F04F7C
S3150800470C9946002385B08A46C9F8003003A9144691
S3150800471C0546FEF779FC8046002839D195F81180B4
S3150800472CB8F1000F34D12B7CD80773D56B69EF68B9
S3150800473CFF1AA74228BF274657B305F1280BC3F320
S3150800474C0801002946D103994A89013A12EA5322EB
S3150800475C57D0A8694B690238023B984274D24B89E8
S3150800476C8E6A03FB0066002E6ED07C0A164413D0A4
S3150800477C1019984288BF9C1A4878234632465146E7
S3150800478CFDF7D4F8002848D04FF0010885F81180B9
S3150800479C404605B0BDE8F08FEA69B24216D02B7CCC
S315080047AC48785B060BD501235946FDF70BF900280B
S315080047BCEAD12B7C039A23F040032B7450780123FF
S315080047CC32465946FDF7B2F80028DDD16969EE6123
S315080047DCC1F30801C1F50074BC4228BF3C46283118
S315080047EC294422465046FEF731FC6B69D9F800205D
S315080047FC234422443F1B6B61A244C9F800209ED176
S3150800480CC6E7D3B9A86801281ED9411CBCD00399A0
S3150800481CA8619FE74FF00708BAE72B7C5A060AD51A
S3150800482CE869801BA04206D20AEB40204FF40072BE
S3150800483C5946FEF70BFC6402D7E7A969286801926A
S3150800484CFEF78CFE019ADEE74FF0020885F8118018
S3150800485C9EE700BF2DE9F04F9A46002385B08B469C
S3150800486CCAF8003003A916460446FEF7CDFB804667
S3150800487C002853D194F81180B8F1000F4ED1227C40
S3150800488C910740F18C806369F34200D3DE43002E16
S3150800489C73D004F128020192C3F3080000284BD107
S315080048AC039AB2F80A9009F1FF3919EA53290FD17C
S315080048BC002B7DD1A068002800F08280012800F02A
S315080048CC9D80421C26D0A368A061039A03B9A060F8
S315080048DC237C5B0655D4A7695369023F023B9F426A
S315080048EC80F08C805389916A03FB0717002F00F020
S315080048FC8580750A4F4415D009EB0501994288BF86
S3150800490CA3EB090550782B463A465946FDF75AF853
S3150800491C002847D04FF0010884F81180404605B0AE
S3150800492CBDE8F08FE3696069BB4202D0E368834255
S3150800493C4ED8E761C0F30800C0F50075B54228BF2C
S3150800494C3546283020442A465946FEF77FFB237CF9
S3150800495C43F0400323746369E2682B449A4238BFD8
S3150800496C1A461146DAF80020761B2A446361E16080
S3150800497CAB44CAF800208FD1227C42F02002227464
S3150800498CCCE750780123E2690199FDF71BF800285A
S3150800499CC0D1237C039A23F0400323749BE74FF082
S315080049AC0708BBE7E169C91BA9421BD36D02D2E70D
S315080049BCA1692046FEF732FF00287FF47FAFDBE7BC
S315080049CC49462046FEF72AFF00287FF477AFD3E73F
S315080049DC507801233A460199FCF7A8FF002899D18B
S315080049EC6069A6E70BEB41214FF400720198FEF7BC
S315080049FC2DFB237C23F040032374D7E74FF00208E2
S31508004A0C84F811808AE700BF70B50A2982B00E4671
S31508004A1C05461AD06C68002C08DB2B1901343C2C83
S31508004A2C1E7305DCAB686C600133AB6002B070BDFD
S31508004A3C01AB224605F10C012868FFF70BFF019B19
S31508004A4C1C1B18BF4FF0FF34ECE70D21FFF7DCFFFA
S31508004A5CE0E700BFF0B583B001A90446FEF7D4FA27
S31508004A6C002839D1237C9A0636D55B06019D3CD4A1
S31508004A7C216AEB6A994231D1636ADA7A42F02002EA
S31508004A8CDA72A2682168C2F30720D8769A76097872
S31508004A9C032903D1120C110A1A75597500214820DD
S31508004AAC61270126E26858764FEA122C1A7783F8A2
S31508004ABC1DC04FEA124C120E997583F81EC0DA7790
S31508004ACCD9759974D9741F762846EE70FEF7EEFAE6
S31508004ADC237C23F02003237403B0F0BD2846FEF78D
S31508004AEC4BFB0028F8D1019DC6E768780123E269DB
S31508004AFC04F12801FCF766FF28B9237C019D23F0F5
S31508004B0C40032374B4E70120E6E700BF10B582B072
S31508004B1C0446FFF79FFF08B102B010BD01A9204655
S31508004B2CFEF772FA0028F7D1206002B010BD00BF5C
S31508004B3C2DE9F04182B00F4601A90446FEF764FA46
S31508004B4C054600284DD1657C002D4AD1E368BB4249
S31508004B5C04D2227C12F0020F08BF1F46002263699A
S31508004B6C6261002F3DD0019AB2F80A804FEA4828B4
S31508004B7C3BB1013B7A1EB3FBF8F1B2FBF8F28A4261
S31508004B8C57D2A668002E60D0A661002E30D1636974
S31508004B9CC3F30802002A56D0E269B24253D0237CEA
S31508004BAC01995B06487804F128070AD5012339468A
S31508004BBCFCF708FFC8B9237C019A23F04003237439
S31508004BCC5078394601233246FCF7B0FE68B963695A
S31508004BDCE268E661934204D9227CE36042F0200342
S31508004BEC2374284602B0BDE8F08101256574F8E700
S31508004BFC474513D84CE02046FEF710FE064678B318
S31508004C0C721CF2D0012E1BD9019B5B69B34217D9D2
S31508004C1C6369B8454344A661636123D2237CA7EB39
S31508004C2C080798073146E6D42068FEF797FC06462F
S31508004C3CE6E7C8F1000213406361FF1AA669A4E708
S31508004C4C02256574CDE7E268C4E731462046FEF7CF
S31508004C5CE5FD01280646F3D0431CC6D0A06093E7B1
S31508004C6C474663693B44C7F30802636172B101990D
S31508004C7CB01E4A69023A9042E2D24E898A6A00FB11
S31508004C8C0626002EDCD006EB572681E716467FE76C
S31508004C9C6369E7E730B591B001900D46002205A986
S31508004CAC01A8FEF7C1FA044610B1204611B030BD72
S31508004CBC0E4A02AB019905A80F920D93FFF79EF9C0
S31508004CCC04460028F1D10D9B93F90B30002B0ADB17
S31508004CDC002DEAD00B9BA875002BE6D0294605A813
S31508004CECFFF7E6FAE1E70624DFE700BF780F0020B6
S31508004CFC30B59DB00190022202A901A8FEF794FADC
S31508004D0C029B069308B11DB030BD254A03AB06A815
S31508004D1C019910920E93FFF771F90028F3D10E9BA7
S31508004D2C93F90B30002B05DB9DF81E30DA0703D5FB
S31508004D3C0720E8E70620E6E7029D0D9A2978D07E3B
S31508004D4C947E032944EA00240BD0DB0610D406A86B
S31508004D5CFEF760FE0028D6D1D4B90298FEF7A6F95C
S31508004D6CD1E7517D127D42EA012244EA0244ECE77E
S31508004D7C11A8002111951394FEF766FC0028C2D1E0
S31508004D8C11A8FFF715FB0028D2D00428BBD1DEE703
S31508004D9C0246214606A8FFF7EDF80028DDD0B2E753
S31508004DAC780F00202DE9F041804617460546002469
S31508004DBC82B04E1EB44212DA01AB0122694638465D
S31508004DCCFFF79CFC019B012B09D19DF800300D2B9C
S31508004DDCF0D00A2B05F8013B04F10104EAD10023B3
S31508004DEC9C4214BF404618462B7002B0BDE8F081B1
S31508004DFC10B5044600230846217894B0CDE9010382
S31508004E0C0393B1B101A8FFF7FFFD14F8011F0029A0
S31508004E1CF8D1029A002A0EDB01986B4604A9FFF713
S31508004E2C19FD40B9029A009B9A4204D1039814B012
S31508004E3C10BD0A46F1E74FF0FF30F8E77F2819D97D
S31508004E4C89B910B40E4AC72303E0802915D032F865
S31508004E5C023F98428CB201F10101F6D104F18000AF
S31508004E6C80B210BC7047FF2805D8054B803833F83C
S31508004E7C100070477047002070470020F1E700BF0C
S31508004E8C80530008284AB0F5805F284B41F67D51BF
S31508004E9C3CBF134661210433002943D0814241D8D3
S31508004EAC70B433F8022C1E46D4B26518A8424FEAE1
S31508004EBC122208DB04337AB133F8041C09B1814297
S31508004ECCEFD970BC7047082AFBD8DFE802F00F133D
S31508004EDC191C1F2225280B0006EB440336F8141060
S31508004EEC0433EBE7A0F5E35080B2EAE7411A33F84E
S31508004EFC1100E6E7411A01F00103C01A80B2E0E797
S31508004F0C103880B2DDE7203880B2DAE7303880B264
S31508004F1CD7E71A3880B2D4E7083080B2D1E75038D0
S31508004F2C80B2CEE7704700BF80540008745600085C
S31508004F3C70B500250C4E0D4CA41BA410A54209D126
S31508004F4C00F050F800250A4E0A4CA41BA410A542E2
S31508004F5C05D170BD56F8253098470135EEE756F859
S31508004F6C253098470135F2E73C5800083C580008AC
S31508004F7C3C58000840580008044B054A1B681B6A35
S31508004F8C002B08BF1346D3F8EC007047100000201E
S31508004F9C7400002082B001B901A942B14BB1137853
S31508004FAC0B601278101C18BF012002B0704710460F
S31508004FBCFBE76FF00100F8E703460244934200D181
S31508004FCC704703F8011BF9E749B1FF2A8BBF8A23FF
S31508004FDC0A700360012088BF4FF0FF3070470846FF
S31508004FEC70470000F8B500BFF8BC08BC9E46704771
S31108004FFCF8B500BFF8BC08BC9E4670471C
S315080050082F626F6F746C6F672E74787400000000D7
S315080050182F64656D6F70726F675F6F6C696D657801
S315080050285F73746D3332703130332E737265630073
S315080050380000000000000000010203040607080932
S315080050480000000001020304433A2F576F726B2FC2
S31508005058736F6674776172652F4F70656E424C542C
S315080050682F5461726765742F536F757263652F4184
S31508005078524D434D335F53544D333246312F636196
S315080050886E2E6300050206020603070308030903D2
S3150800509809040A040B040C040C050D050E050F0576
S315080050A80F06100610071008433A2F576F726B2F12
S315080050B8736F6674776172652F4F70656E424C54CC
S315080050C82F5461726765742F536F757263652F4124
S315080050D8524D434D335F53544D333246312F727315
S315080050E83233322E6300000008000000000000007A
S315080050F8303A0000433A2F576F726B2F736F6674F6
S31508005108776172652F4F70656E424C542F546172E1
S315080051186765742F536F757263652F66696C652E9C
S31508005128630000004669726D776172652075706460
S315080051386174652072657175657374206465746534
S31508005148637465640A0D00004F70656E696E6720A2
S315080051586669726D776172652066696C6520666F27
S31508005168722072656164696E672E2E2E0000000033
S315080051784552524F520A0D004F4B0A0D00000000C7
S315080051885374617274696E67207468652070726FEB
S315080051986772616D6D696E672073657175656E6393
S315080051A8650A0D0050617273696E67206669726DCB
S315080051B8776172652066696C6520746F206465740A
S315080051C865637420657261736520626C6F636B73BF
S315080051D82E2E2E0045726173696E67200000000046
S315080051E82062797465732066726F6D206D656D6FC0
S315080051F87279206174203078000000005265616475
S31508005208696E67206C696E652066726F6D206669BF
S315080052186C652E2E2E4552524F520A0D000000007C
S31508005228496E76616C696420636865636B73756D2E
S3150800523820666F756E642E2E2E4552524F520A0DF1
S315080052480000000050726F6772616D6D696E6720A5
S315080052580000000020627974657320746F206D65FC
S315080052686D6F7279206174203078000057726974FE
S31508005278696E672070726F6772616D20636865630F
S315080052886B73756D2E2E2E00436C6F73696E6720CF
S315080052986669726D776172652066696C650A0D00C4
S315080052A84669726D776172652075706461746520E8
S315080052B87375636365737366756C6C7920636F6D54
S315080052C8706C657465640A0D000000004F70656EA1
S315080052D8424C5400809A45418E418F804545454940
S315080052E849498E8F9092924F994F555559999A9B3D
S315080052F89C9D9E9F41494F55A5A5A6A7A8A9AAABB7
S31508005308ACADAEAFB0B1B2B3B4B5B6B7B8B9BABB4F
S31508005318BCBDBEBFC0C1C2C3C4C5C6C7C8C9CACB3F
S31508005328CCCDCECFD0D1D2D3D4D5D6D7D8D9DADB2F
S31508005338DCDDDEDFE0E1E2E3E4E5E6E7E8E9EAEB1F
S31508005348ECEDEEEFF0F1F2F3F4F5F6F7F8F9FAFB0F
S31508005358FCFDFEFF01030507090E10121416181C9A
S315080053681E000000222A3A3C3E3F7C7F00000000CF
S315080053782B2C3B3D5B5D0000C700FC00E900E20002
S31508005388E400E000E500E700EA00EB00E800EF00CB
S31508005398EE00EC00C400C500C900E600C600F4002B
S315080053A8F600F200FB00F900FF00D600DC00A200B8
S315080053B8A300A500A7209201E100ED00F300FA007A
S315080053C8F100D100AA00BA00BF001023AC00BD0046
S315080053D8BC00A100AB00BB009125922593250225A8
S315080053E824256125622556255525632551255725E2
S315080053F85D255C255B251025142534252C251C25BB
S3150800540800253C255E255F255A25542569256625E8
S31508005418602550256C256725682564256525592541
S315080054285825522553256B256A2518250C258825C0
S3150800543884258C2590258025B103DF009303C003B6
S31508005448A303C303B500C403A6039803A903B403B7
S315080054581E22C603B50329226122B10065226422E9
S3150800546820232123F7004822B0001922B7001A2260
S315080054787F20B200A025A00061001A03E0001703E8
S31508005488F8000703FF000100780100013001320126
S315080054980601390110014A012E0179010601800128
S315080054A84D0043028101820182018401840186013B
S315080054B88701870189018A018B018B018D018E017C
S315080054C88F0190019101910193019401F6019601CA
S315080054D89701980198013D029B019C019D012002B4
S315080054E89F01A001A001A201A201A401A401A6018D
S315080054F8A701A701A901AA01AB01AC01AC01AE013C
S31508005508AF01AF01B101B201B301B301B501B501EC
S31508005518B701B801B801BA01BB01BC01BC01BE019B
S31508005528F701C001C101C201C301C401C501C40113
S31508005538C701C801C701CA01CB01CA01CD011001BB
S31508005548DD0101008E01DE011201F3010300F101FC
S31508005558F401F401F8012801220212013A020900AD
S31508005568652C3B023B023D02662C3F024002410283
S31508005578410246020A01530240008101860155028A
S3150800558889018A0158028F015A0290015C025D025C
S315080055985E025F0293016102620294016402650277
S315080055A866026702970196016A02622C6C026D020E
S315080055B86E029C01700271029D01730274029F01BA
S315080055C876027702780279027A027B027C02642CD8
S315080055D87E027F02A60181028202A901840285024F
S315080055E886028702AE014402B101B20145028D0264
S315080055F88E028F0290029102B7017B030300FD0316
S31508005608FE03FF03AC0304008603880389038A03A1
S31508005618B1031103C2030200A303A303C4030803C7
S31508005628CC0303008C038E038F03D8031801F203F7
S315080056380A00F903F303F403F503F603F703F7037C
S31508005648F903FA03FA033004200350041007600428
S3150800565822018A043601C1040E01CF040100C004E0
S31508005668D004440161052604000000007D1D0100E0
S31508005678632C001E9601A01E5A01001F0806101F5B
S315080056880606201F0806301F0806401F0606511F73
S315080056980700591F521F5B1F541F5D1F561F5F1FA8
S315080056A8601F0806701F0E00BA1FBB1FC81FC91F38
S315080056B8CA1FCB1FDA1FDB1FF81FF91FEA1FEB1FCC
S315080056C8FA1FFB1F801F0806901F0806A01F08065A
S315080056D8B01F0400B81FB91FB21FBC1FCC1F01009A
S315080056E8C31FD01F0206E01F0206E51F0100EC1FB4
S315080056F8F21F0100FC1F4E21010032217021100201
S31508005708842101008321D0241A05302C2F04602C0B
S315080057180201672C0601752C0201802C6401002DF4
S31508005728260841FF1A0300004300504F5349580002
S315080057382E00002020202020202020202828282865
S31508005748282020202020202020202020202020203B
S31508005758202020881010101010101010101010108B
S31508005768101010040404040404040404041010109B
S315080057781010101041414141414101010101010147
S3150800578801010101010101010101010101011010D5
S31508005798101010104242424242420202020202021B
S315080057A802020202020202020202020202021010A7
S315080057B81010200000000000000000000000000093
S315080057C800000000000000000000000000000000C3
S315080057D800000000000000000000000000000000B3
S315080057E800000000000000000000000000000000A3
S315080057F80000000000000000000000000000000093
S315080058080000000000000000000000000000000082
S315080058180000000000000000000000000000000072
S315080058280000000000000000000000000000000062
S30908005838000000005E
S3090800583C3101000820
S309080058400D01000840
S315080058440024F40001000000100000000104000018
S315080058541400002000000000000000000000000002
S315080058640000000000000000000000000000000026
S315080058740000000000000000000000000000000016
S315080058840000000000000000000000000000000006
S3150800589400000000000000000000000000000000F6
S315080058A400000000000000000000000000000000E6
S315080058B40000000043000000000000000000000093
S315080058C400000000000000000000000000000000C6
S315080058D40000000043000000000000000000000073
S315080058E400000000000000000000000000000000A6
S315080058F40000000043000000000000000000000053
S315080059040000000000000000000000000000000085
S315080059140000000043000000000000000000000032
S315080059240000000000000000000000000000000065
S315080059340000000043000000000000000000000012
S315080059440000000000000000000000000000000045
S3150800595400000000430000000000000000000000F2
S315080059640000000000000000000000000000000025
S3150800597400000000430000000000000000000000D2
S315080059840000000000000000000000000000000005
S3150800599400000000D54F0008A14F000800000000D1
S315080059A43A57000838570008395700083957000885
S315080059B43957000839570008395700083957000875
S315080059C4395700083957000839570008FFFFFFFF01
S315080059D4FFFFFFFFFFFFFFFFFFFF0000010041532A
S315080059E443494900000000000000000000000000D0
S315080059F40000000000000000000000000000415301
S31508005A0443494900000000000000000000000000AF
S31508005A140000000000000000000000000000000074
S7050800067973
